:030000000219FDE5
:03000B000200AA46
:03002B0002015679
:03005B000202E5B9
:030073000202D2B4
:1000800002030406080C10182030406080040608A3
:100090000C10182030406080A0C00003070F1F0D17
:1000A0000D04050D050205030302C2AFC0D0C0E078
:1000B000206214E5256009E473E525F4F58AD2622F
:1000C000D0E0D0D0D2AF3285268AC262E526F46075
:1000D00029D0E0D0D0D290D291D292D2AF32D29069
:1000E000D291D292206F0C206509740AD5E0FDE50B
:1000F0007B4290D0E0D0D0D2AF32758A00C28DD290
:100100006201F301B9306805206502C29001B9307F
:100110006805206502C29101B9306805206502C2F8
:100120009201B9C29330680A2065077428D5E0FDB2
:10013000C29001B9C29430680A2065077428D5E0DE
:10014000FDC29101B9C29530680A2065077428D5AF
:10015000E0FDC29201B9C2AFC2AD53E6EFC0D0C05C
:10016000E0D2D3D2AFC2CEE52A600720744F152A61
:1001700021BD7800790020742EE580307E01F430B6
:10018000E70278FF53DACF207E0343DA20307E0384
:1001900043DA10C2D8C271E580307E01F430E70244
:1001A00079FFC3E89970CB306103752A1820740376
:1001B000752A18885CD270E86003755F0020740DA2
:1001C000E52B6004152B21CD43DA01C2D820700243
:1001D000413CA85C206102C2702074367982B70469
:1001E00031C3E894F0400374F0F8E8C4540F28F8E1
:1001F0007984B703024112C313C313872120080275
:10020000C313200A06C3C898F8411228F850037493
:10021000FFF88822E52D54066022206B1FE536C3C7
:1002200033C333F8E564C313C313F9C39522400203
:100230008922E82522F52250037522FF7882B60430
:100240004E852224A824C3E52495614002A861C3F9
:10025000E895634002A8638825E5667002418DC376
:10026000E8AA669A5003E8FAE4F9EAC333FBE568C2
:10027000F45B29400D2567F8E56760021567400BC0
:10028000418D0AC3E5679A5002056778FF882620EA
:10029000CF0AD0E0D0D043E610D2AD32C2CF053A7B
:1002A0007801E52A6005307402152AC3E55C9401E3
:1002B0004005755F0041C8756000756900E55F2401
:1002C00001F55F5003755FFFD0E0D0D043E610D258
:1002D000AD32C2AF53E67F7592FA7593FFC2607577
:1002E0009104D2AF32C2AF53E6EFC2ADC0D0C0E08E
:1002F000C0F0D2D3D2AFA8FBA9FCC2D83071026142
:100300004C53DACF207E0343DA10307E0343DA20E9
:10031000D271E580307E01F420E7026123882789CD
:1003200028A17953DACF207E0343DA20307E0343BD
:10033000DA10C2D8C271307402A1657800E580304D
:100340007E01F430E702A165885CA14D53DACF202D
:100350007E0343DA20307E0343DA10C2712061024B
:10036000812553DACF207E0343DA10307E0343DA4F
:1003700020C2D8D27188578958C3E89555F8E995B5
:1003800056F97B007E087A00C3E8948CE99400500B
:1003900005755B008117882178A2E6A8216055C306
:1003A000E894C8E994005008E4D2E4FB7A0A61F2C8
:1003B000C3E89468E994015008E4D2E3FB7A0F6142
:1003C000F2C3E894D0E994025008E4D2E2FB7A1E2A
:1003D00061F2C3E894A0E994055008E4D2E1FB7A05
:1003E0003C61F2C3E89498E994085008E4D2E0FB39
:1003F0007A787E00C3E89559FCE9955AFD30E70A02
:10040000ECF42401FCEDF43400FD755B00C3EC9AC0
:10041000ED9E5003755B018859895A85575585585B
:10042000567802A14DC3E89527F8E99528F9307C64
:1004300002A131307B02A131307A02A12A2075025B
:100440008148E9FDE8FC8167E9C313F9E813F83056
:100450007902A12AE9C313F9E813F8307802A12A36
:10046000E9C313FDE813FC20612CC3EC941CED944C
:0E047000024002817EED701EC3EC94C850184D
:10047E000529E52970021529C3E529940A5002A120
:10048E0065755C00D270A165E52960021529788832
:10049E00E6F97400207F087896B90302789EE62468
:1004AE00FAFEE43400FFC3EC9EFCED9FFD9208B90A
:1004BE000310A2085007207609D27681D03076023A
:1004CE00C276A2085016B9030DECF42401FCEDF42B
:1004DE003400FD0204EA78007900A131B90315EC6D
:1004EE0033FCED33FDC3EC940AFCED9400FD500497
:1004FE007C007D00C3EC94FFED9400400678FF79FC
:10050E0000A131EC8572F0A4C5F0A2F733F87900A2
:10051E00400302054D78FF790002054DE9C313F93A
:10052E00E813F8307C0EE9600278FFC3E81338F860
:10053E00E43400F9C3E894FFE99400400278FF88A0
:10054E005CD270206102A165741FF4552F4BF52FFC
:10055E00C274EB7002D274752A18307403752A0AAD
:10056E00306102A17920740353DAFE207403752BD7
:10057E0006D0F0D0E0D0D0D2AD43E61032790102F1
:10058E0005A979030205A9790A0205A9791E0205B2
:10059E00A979640205A979C80205A97817E4D5E0FE
:1005AE00FDD8FAD9F6227A147B780205D07A107B20
:1005BE008C0205D07A0D7BB40205D07A0B7BC80273
:1005CE0005D0E573D5E001227902E4C294D5E0FDB1
:1005DE00C291D5E0FDD291D5E0FDD294D5E0FDE9F2
:1005EE0020E002C29030E002C292E573D5E0FDE950
:1005FE0020E002D29030E002D2927496D5E0FDD97E
:10060E00C9EAF8D5E0FDD8FBDBB8C29422C37C0062
:10061E007D0075F00005F0EA33FAEB33FB50F6EB94
:10062E0013FBEA13FAC3E9FFE8FEE89AF8E99BF92F
:10063E005004EFF9EEF8B3EC33FCED33FDD5F0DFFB
:10064E00EDF9ECF822E889F08A20D2D4F8A9F07BF3
:10065E000030F70B7BFFF42401F8E9F43400F9E8DD
:10066E008520F0A4ADF0F8E98520F0A4AFF0FEED02
:10067E002EF974003FFA7C04C3EA13FAE913F9E881
:10068E0013F8DCF48BF030F70AE8F42401F8E9F4FF
:10069E003400F9E889F0C2D4F8A9F0227882B604C1
:1006AE0003020705C3E55C940140030206CF8522D1
:1006BE0024E4F544F545F546F547F548C26E0207C4
:1006CE00057882E6FCD26EE522F523783879C7AA42
:1006DE0040AB41C3EB13FBEA13FAEC146013C3EB0C
:1006EE0013FBEA13FAEC14146007C3EB13FBEA13C3
:1006FE00FAD11B8844894522C3E5449523F8E54584
:10070E009400F9500CC3E89480E994FF4016020758
:10071E0036C3E8947FE994005003020736787F7958
:10072E0000020736788079FF8849894A22E54925F3
:10073E0046F8E54A3547F9854A20E4300701F43595
:10074E0048FA30E709C3EA94F04015020774C3EA89
:10075E00940F500302077478FF79FF7A0F02077423
:10076E00780079007AF0C3E5249561500AC37401CC
:10077E009524500B020792E54A20E70E020792E5F8
:10078E004A30E706884689478A482278A5E6FAC3A2
:10079E00E54933F8E54A33F9D153E930E70BC3E8BD
:1007AE009480E994FF4013E1CCC3E8947FE9940070
:1007BE005002E1CC787F7900E1CC788079FFE82097
:1007CE00E715C3E52398F84009C3E89401400302F6
:1007DE0007F378010207F3E8F424012523F8400318
:1007EE000207F378FF884B2278A6E6FAA847A948B5
:1007FE00120653E930E70CC3E89401E994FF401662
:10080E00020828C3E894FFE99400500302082878F0
:10081E00FF7900020828780179FFE920E715C3E582
:10082E004B98F84009C3E89401400302084F780141
:10083E0002084FE8F42401254BF8400302084F78D4
:10084E00FF88242278FF20692879A1E76023E541FB
:10085E00601F74FF8541F0848539F0306A0375F0AE
:0F086E0005A4F8C5F0600278FFC3E89564500256
:10087D00A864886322C3E5409440E5419401E56393
:10088D005003140193046002F5632202089B227544
:10089D00E890227883E6FF30EDF9A8BDA9BE05707A
:1008AD00C3E57094084052757000E9FA79A0E760CD
:1008BD0044EA7007E571601B0208D4C3E8957160C6
:1008CD0010E5715006600C140208E00460F902088E
:1008DD00E0E571F571C3946D401B7561C0C394045F
:1008ED004013756180C39404400B756140C394043B
:1008FD00400375610075BB0622E56124105002743A
:10090D00FFF5617982B70402212DC3A861E5249812
:10091D005002A824C3E895634002A8638825882661
:10092D00E570B4070375BB1022743279A787F0A464
:10093D00C5F0A2F733F8C3E895614002A86188229B
:10094D008824882588268864227540007541F02208
:10095D00C2AF75C820A8CCA9CDAA3A30CF010A756F
:10096D00C824D2AFAB3BAC3C883B893CC3E89BF879
:10097D00E99C206908F9306602416E21C8AD3D8AB7
:10098D003DF9EA9DFA600678FF79FF21ADAE3EAFE5
:10099D003F8B3E8C3FA83BA93CC3E89EF8E99FF9ED
:1009AD00C3E54113FBE54013FAE82AF540E93BF5B1
:1009BD004150067540FF7541FF4115AA40AB41AC52
:1009CD0040AD417E047F02C3EB9404400D1E1FC356
:1009DD00EB94084005206A021E1FC3ED13FDEC13B6
:1009ED00FCDEF7C3EA9CFAEB9DFBEF6009C3E9134C
:1009FD00F9E813F8DFF7EA28FAEB39FB8A408B4167
:100A0D0050067BFF8B408B41C3EB94025002D266A4
:100A1D003069047F0341407892E6FFC3E537948245
:100A2D0040110FC3E53794A040010FC3EF9406406A
:100A3D00027F057E02E541C4540FF9E541C454F02F
:100A4D00F8E540C4540F28F8C3E89EFAE99400FB7A
:100A5D004009C3EA9402EB940050047A02E4FB418E
:100A6D00BAAA40AB41EBC4FEEAC4540F4EFCC3EA34
:100A7D009CFAEB9400FBC3E813C313F8EA28FAEBD6
:100A8D003400FB8A408B41C3EB94024002C266786E
:100A9D0002EBC4FE7B00EAC4540F4EFAC3EA98FA87
:100AAD004005C3940250027A027892E6FF3060024C
:100ABD0041BA855192855293D26043E680C3E49A40
:100ACD00F8E49BF93066026146E8FAE9FBD3E913D5
:100ADD00FDE813FC88518952C3EF94036038EF2071
:100AED00E00DE82CF8E93DF9ECFAEDFB020B0FE80F
:100AFD0028F8E939F9C3E82402F8E93400F97AFE57
:100B0D007BFFC3EF9403400E8A538B54884D894E5F
:100B1D008C4F8D50617A885389548A4D8B4E8C4FF2
:100B2D008D503069127553F07554FF754FF0755037
:100B3D00FF7551F07552FF617AE8FAD3E813FC881E
:100B4D0051C3EF94036020EF20E007E82CF8ECFA96
:100B5D006166E8282402F87AFEC3EF940340088A00
:100B6D0053884D8C4F617A88538A4D8C4FE568C3FD
:100B7D00335002646BF5683060026184753402D2C3
:100B8D006043E680E52D54066034A840A941C3E9D1
:100B9D0013F9E813F8C3E913F9E813F8306904E918
:100BAD002440F9C2AF53E67F759100C3E498F594E4
:100BBD00E499F595759104D26043E680D2AF22D2C7
:100BCD0064754300752000306C03752040020BEBFB
:100BDD00D264754300752040306C03752000780198
:100BED007901206620E52D54066002C2647914E572
:100BFD0041C313700104F8C3941440027814306992
:100C0D0004781B791B206010E543600C306903D517
:100C1D003404D26D8196718C0543E59BF45440B537
:100C2D002002818030690908C3E8994001188112BA
:100C3D0020640A08C3E899400261EB8112C264C2C4
:100C4D00AF53E67F7591003066127594007595F877
:100C5D00759104D26043E680D2AF61EBE5417EFF32
:0F0C6D00C3334005C3334001FEC3E49E759400BA
:100C7C00F595815DC3E5339401500261EB3064025C
:100C8C0061EBD80281948112C26DC2AF53E67F75BD
:100C9C009100855394855495759104854D92854E9C
:100CAC0093D26043E680D2AFE52D54066008206AEB
:100CBC00020533020CD2306D0D206C0A206407152E
:100CCC008115810215852278003064027801E537A0
:100CDC0075F007A4F9E5F028F5F0E9A2F013A2F1FC
:100CEC0013A2F213F537C394785003753778C3E524
:100CFC003795384008D265D290D291D292306002AA
:100D0C00A109854F92855093D26043E68022207DC5
:100D1C0016C2AF754202C294D293306202C292D212
:100D2C00AF759F11020F0AC2AF754202C294D295E1
:100D3C00306202C290D2AF759F11020F0A3072431B
:100D4C00207D20C2AF754203900134757B10D29286
:100D5C00C295306204C291A167D294D2AF759F2123
:100D6C00020F0AC2AF754203900134757B10D2900A
:100D7C00C293306204C291A187D294D2AF759F0105
:100D8C00020F0A207D17C2AF75420390010FD29259
:100D9C00306202C291D2AF759F21020F0AC2AF75A9
:100DAC00420390010FD290306202C291D2AF759F74
:100DBC0001020F0A207D16C2AF754204C293D29570
:100DCC00306202C291D2AF759F01020F0AC2AF7599
:100DDC004204C295D293306202C291D2AF759F2168
:100DEC00020F0A307243207D20C2AF75420590017C
:100DFC0023757B08D291C294306204C290C10DD28B
:100E0C0093D2AF759F11020F0AC2AF7542059001C4
:100E1C0045757B20D291C294306204C292C12DD20E
:100E2C0095D2AF759F11020F0A207D17C2AF754284
:100E3C0005900105D291306202C290D2AF759F111C
:100E4C00020F0AC2AF754205900119D2913062EBC4
:100E5C00C292D2AF759F11020F0A207D16C2AF75D8
:100E6C004206C295D294306202C290D2AF759F21D5
:100E7C00020F0AC2AF754206C293D294306202C20C
:100E8C0092D2AF759F01020F0A307244207D20C2AE
:100E9C00AF754201900145757B20D290C2933062B0
:100EAC0004C292C1B3D295D2AF759F01020F0AC290
:100EBC00AF754201900123757B08D292C2953062C6
:100ECC0005C290020ED4D293D2AF759F21020F0AA5
:100EDC00207D17C2AF754201900119D29030620289
:100EEC00C292D2AF759F01020F0AC2AF7542019038
:100EFC000105D292306202C290D2AF759F21C265B9
:100F0C0022900103757B00D290D291D292C293C2EF
:100F1C0094C295C262227880760908760908760414
:100F2C000876FF0876030876FF087609087601082C
:100F3C007601087601788C76010876FF0876FF0832
:100F4C0076FF0876FF0876FF0876030876FF0876AA
:100F5C00FF0876FF0876250876D0087628087650A4
:100F6C000876040876FF08760208760008767A0878
:100F7C0076FF087601087601087600087603087675
:100F8C0000227887E6FFC2727888E6C39403600873
:100F9C00C27DE630E102D27DC27E7889E630E10284
:100FAC00D27EC3EF94026008758E01D273020FC11A
:100FBC00758E00C273227880E6149000809378A519
:100FCC00F67881E6149000809378A6F67886E6147D
:100FDC0090008D9378A7F67886E6F539C394025085
:100FEC0003753902789CE67538FFB402037538A096
:100FFC00B4030375388278A3E61490009A93F566CF
:10100C00120F0D22227896E6FA7897E6FB7888E69E
:10101C00B40305C3EB940EFB307F047A007BFFC353
:10102C00EB9AFCC3948250027C827572000572ECC0
:10103C008572F0A4C3E5F0947D40F222D27F1111A9
:10104C0012059A12059A7A007B007C10120590E525
:10105C005C2AFA74003BFBDCF37C04C3EB13FBEA65
:0D106C0013FADCF7FEC27F111122757C0023
:10107900757D00E5EF20E6037520000520903FFF10
:10108900E520146006901DFF146000930460037549
:10109900EF1653D9BF7581C043FF8012058B75EFD9
:1010A9000643B203E5B3240220E70DF521E5E32069
:1010B900E0068521B343E301120F0D7580FF75A486
:1010C9000075F19175D47F75900775A53F75F2FF8D
:1010D90075D50075A60175E241120F0DE4F8F6D831
:1010E900FD756801120F221215D67898867375302E
:1010F90001C2AF1205A41205B412059A1205BB125A
:10110900059A1205C212059AC2AF757C00757D0059
:1011190078FA79FA308707D9FBD8F7021C00120F41
:101129008E120FC21110111178988673120F0D7556
:10113900881075890275C82475910475D84075A8F9
:101149002275B80275E690759B80759D0075D10E64
:1011590075BC5875BB0675BA1175E88012058BD236
:10116900AF12089875360053DACF207E0343DA2090
:10117900307E0343DA1043DA01C2D8C2711205A4E2
:10118900D2617B037A0CE55B70077A0CDB030211F1
:101199001112059A207003021111C270E55CC39403
:1011A9000240E1E52F541F855E5DF55EB55DD5DA38
:1011B900D5C26153DACF207E0343DA20307E034360
:1011C900DA10C2D8C27178A2E67008D274E52F5439
:1011D900E0F52FC27575290012059F307409C3E522
:1011E90029940A4002D27512059078023074027867
:1011F90000C3E55C9840F0C2AF1205B41205B41201
:1012090005B4D2AF1205A4754C007888E6B4030280
:101219006106120590788CE6C39401500302130607
:10122900E530C394015003021306757CA5757DF161
:10123900207435C3E55C94FF5003021306C2AF1254
:1012490005C9D2AF12059FC3E55C940150EFC2AF47
:101259001205B41205951205B4D2AF12059FC3E564
:101269005C94FF40E902178E7F02D27F11111205AB
:101279009FC2AFC27F1111AE5CC3E55C947FD2AF50
:101289005002611612058BC2AF1205C9D2AFDFDA5F
:101299001148C3EE7897F61205A41217117F0AD2E6
:1012A9007F111112059FC2AFC27F1111AE5CC3E558
:1012B9005C947FD2AF50E612058BC2AF1205B4120F
:1012C90005951205B4D2AFDFD61148EE24037896FE
:1012D900F6F87997E7C394824003985006E8248288
:1012E9007897F61205A412162412174012059F11B9
:1012F90011C3E55C94FF5002413302178E757C00DF
:10130900757D00C3E55C954C4003855C4C12059FD7
:1013190078017988E7B403027805C3E55C9840024F
:101329004113C2AF1205C91205C91205C9D2AF12BC
:1013390005A4753000E4F531F5320531E531F47075
:101349003F0532789AE67819146012783214600DE4
:10135900787D14600878FA146003753200C3E532A9
:1013690098401D120F0D12058B15327531007899B1
:101379008673C2AF1205C9D2AF7898867312059FDA
:10138900120595E52A70053074022111780120743F
:10139900027806C3E55C9840A17888E6C3940360A7
:1013A9000312059FE52A7003021111C2AF120F0D36
:1013B900E4F522F523F524F525F526F567D2AF786E
:1013C90085E6C333F565E4F544F545F546F547F596
:1013D90048F570F52CF52DF53775700875BB1012A9
:1013E900058B12089C30EDFDA8BDA9BEE97001F876
:1013F90088711208A075700875BB10120F8EC2AFE4
:101409007561FF120936852261852262852263D2C0
:10141900AF7522017524017525017526018560695D
:10142900756A017888E6B40307C27D307602D27DF9
:10143900D268D269753300120E66120E95120956DA
:1014490012095D12095612095D120956120BDD12B5
:1014590006AA120CD3120D1A12095D120BCC306EAA
:0D14690003120706206603120852306603C6
:10147600120882120CD3120D4912095D120BDD30CF
:101486006E0312073B120CD3120DC012095D120B2C
:10149600CC306E03120799120CD3120DEF12095DB0
:1014A600120BDD306E031207F6120CD3120E661203
:1014B600095D12089C120BCC120CD3120E95120861
:1014C600A012095D30693285646185646285606950
:1014D600756A0179187A0CC3E53399400FC269D24F
:1014E6006A8A358564618564630214FFC3E55C948A
:1014F60001400302145502158D306A25206C22E541
:1015060035147006C26AD26B8155F535C3E55C9415
:101516000140030214557888E6C39403600302155C
:101526008D75360078FA79A4E760027803C3E55F23
:10153600985054307404E52A604D7888E6B4031751
:10154600207D05207607A15D307602A15D206C071F
:10155600D26C856461819478F0306C05856461781D
:1015660020C3E5419850028155306C1BC26CC27D88
:10157600307602D27DD26A75351285646181550551
:1015860036E55C6002A190753600C2AF120F0D7889
:1015960087E6FE7602120F8E7887EEF6E4F522F5E0
:1015A60023F524F525F526F565752C00752D00D255
:1015B600AF12059F120F0D78A4E66006C290C29185
:1015C600C292307409C3E536940440022111613E8B
:1015D600901A0D7820121666E520B4550CA3121643
:1015E60066E520B4AA03021604757CA5757DF11282
:1015F6000F22121624757C00757D00021623901AA0
:101606000378807B0A121666A308DBF9901A0F7816
:101616008C7B19121666A308DBF9901A2822C2AF32
:101626001216A9121686901A00740E12166BA3745F
:101636000912166BA3741512166B901A0378807B29
:101646000A12166AA308DBF9901A0F788C7B191216
:10165600166AA308DBF91216BC12169A901A2822EB
:10166600E493F622E6438F01538FFDFFC3E583948F
:101676001C400122EF857CB7857DB7F0538FFE2293
:10168600438F02438F01857CB7857DB7901A0DF095
:10169600538FFC22901A0D7455D16B901A0E74AAB2
:1016A600D16B227A3079D07820901A40D166E52025
:1016B600F709A3DAF7227A3079D0901A40E7D16B8E
:1016C60009A3DAF922AB74A875BB01027980BB02C3
:1016D600027981BB03027982BB04027984BB0502CD
:1016E6007986BB06027992BB07027987BB08027925
:1016F600A3BB0902799CBB0A027988BB0B027989D4
:10170600E8F7227C051205A4DCFB22C2AF1205B461
:101716001205BB1205C21205C91205951205B412AF
:1017260005BB1205C21205C91205951205B41205AC
:10173600BB1205C21205C9D2AF22C2AF1205C91229
:1017460005C21205BB1205B41205951205C912058C
:10175600C21205BB1205B41205951205C91205C2BF
:101766001205BB1205B4D2AF22AE74AF75C2AF126A
:1017760005B41205B41205B4120595DEF21205C9B8
:10178600120595DFF8D2AF22F111F109F10975744E
:1017960001757501757600F16F7C05AD5C1205A4C7
:1017A600C3ED955C70F5C3E55C9401400AC3E55C46
:1017B60094FF40320217CAD1CBD124F111C2AF75C2
:1017C600EF16F109DCD50576C3E576940350028061
:1017D600C6F1090575E5741490009F93F808C3E5F2
:1017E6007598500280AEF109F1090574C3E5749449
:1017F6000C5002809C120F22121624C2AF75EF16EF
:03180600121709AD
:0319FD000210765F
:101A00000E0915090904FF03FF0901010155AA0187
:101A1000FFFFFFFFFF03FFFFFF25D0285004FF0259
:091A2000007AFF0101000300FF40
:101A400023506F6C61726973546472343041232087
:101A500023424C48454C4923463333302320202031
:101A60002020202020202020202020202020202076
:101C0000C2AFC2D353D9BF7581C043B20343FF8073
:101C1000752438752503B1DC7529A5752AF175E29F
:101C20004043F18053A47F75D4FFD2877DFA7803B7
:101C300079E67C10752200752300901DE97B0675FE
:101C400024987525013087028145208708D8FBD963
:101C5000F9DCF781B7308708D8FBD9F9DCF781B711
:101C6000B19CE493A3C39A6004DDC381B7DBDBB10D
:101C70008E6002812E7B08E493FAA3B16FDBF87AC1
:101C800030B16F752200752300B18EEAFCEBFDC305
:101C9000ED94FE400EB18E8A278B28ED30E0048A49
:101CA000828B83B18E7AC270D8C3ED94FE601950D6
:101CB000CEBD002BEC600F7520007521FF7529004B
:101CC000752A000200008100A827A9280809D80465
:101CD000D90281DCB192EA89AAF281CE0D81A3C337
:101CE000ED94035053EDA2E092007AC5C3E58294CF
:101CF00000E583941C508A200010438F02438F011B
:101D00008529B7852AB7F0300029A827A92808090E
:101D1000438F01538FFDD804D902A133C3E58394C7
:101D20001C4003A3A11689AAE28529B7852AB7F02A
:101D3000A3A116538FFC817F7AC1BD030CE493A34A
:101D4000FAB153DCF8B14B817F8181AA22AB23B178
:101D50006FEBFAEA6222752608C3E52313F523E543
:101D60002213F52250066323A0632201D526EAB18F
:101D7000DCB1DC75260AEAF4200102D287300102C8
:101D8000C287B1DCC3134002C201D526EB22B19257
:101D9000EAFB208702A192308702A197752608AE40
:101DA00024AF25C3EF13FFEE13FEB1E0B1DCC3EAAD
:101DB000133087024480FA30E703632201C3E5232E
:101DC00013F523E52213F52250066323A0632201B5
:101DD000D526D9E52265236523F52222AE24AF2539
:101DE0000E0FDEFEDFFCD20122424C48656C6934E6
:071DF000373164F3300601F6
:00000001FF
